:03000000020355A3
:030003000203E213
:10000600CB30E11520E00FC083C08289828A83CB82
:0C001600F0D082D08322CBF322CBF72263
:10002200ED30E11320E00EC083C08288828C83E031
:10003200D082D08322E2226405700EC083C08288FF
:0B004200828C8393D082D08322E622C0
:10004D00EB30E11320E00EC083C08289828A83E009
:10005D00D082D08322E3226405700EC083C08289D2
:0B006D00828A8393D082D08322E72296
:0A007800E0C0E0A3E0F582D083228F
:09008200E0FBA3E0FAA3E0F9227F
:05008B00C082C08322C9
:10009000E0A3FEE0FFEF8DF0A4CFC5F0CCA42CFCD4
:0900A000EE60038DF0A42CFE2299
:1000A900C2D1C2D5EE30E707D2D1D2D5120156EC72
:1000B90030E705B2D112015E1200D130D10312012D
:1000C9005630D50312015E22BC000EBE0032EF8D00
:1000D900F08420D226FFADF0227B0075F008EF2FC7
:1000E900FFEE33FEEB33FBEE9DEB9C4005FBEE9DF3
:1000F900FE0FD5F0E9E4CECDCBCC227EFF7FFF22E7
:10010900EDB410005022EE8DF084FEEF54F045F06E
:10011900C48DF084C4FCEF540FC445F0C48DF08441
:10012900FFADF0E4CC4FFF22EE8DF08420D2CC7EDF
:1001390008CEC5F0CDCBEF2FFFED33FD10D7079BD0
:100149005005D5F0F1229BFD0FD5F0EA22C3E49FBB
:0D015900FFE49EFE22C3E49DFDE49CFC2219
:040166001201FB2265
:10016A00C0F0C083C082E8C0E0E9C0E0EAC0E0EBCA
:10017A00C0E0ECC0E0EDC0E0EEC0E08E088F09857B
:0E018A00090AE50A24F6600624FD6007800AD3
:10019800120244800C1202448007AE08AF09120311
:1001A8002BAF09D0E0FED0E0FDD0E0FCD0E0FBD0E2
:0F01B800E0FAD0E0F9D0E0F8D082D083D0F02286
:1001C700E4FCFD8EF0ECB5F0068FF0EDB5F00050D5
:0D01D7001AE4FAFBBA0204BB2101D3500761
:0F01E4000BEB70F30A80F00DED70DB0C80D8226E
:0801F30090E002E020E7F92290
:0E01FB0090E002E020E7F990E0007401F022AD
:0E02090090E002E020E7F990E0007402F0229D
:0E02170090E002E020E7F990E000741CF02275
:0E02250090E002E020E7F990E0007418F0226B
:1002330090E002E020E7F9EF5403240490E000F09B
:010243002298
:1002440090E002E020E7F963114090E000E511F04E
:0E02540090E002E020E7F990E000E511F022D2
:1002620090E002E020E7F963114090E002E020E72D
:08027200F990E000E511F02213
:10027A008B0B8A0C890DAB0BAA0CA90D12004D60D1
:01028A002C47
:06028B0012004DB40A0D43
:10029100120244050DE50D701B050C80E2AB0BAAA3
:1002A1000CA90D050DE50D7002050C12004DFF7E28
:0702B1000012032B80C9229B
:1002B8008B0E8A0F8910AB0EAA0FA91012004D6081
:1002C800130510E5107002050F12004DFF7E001295
:0502D800032B80E2226F
:1002DD00E4FE7F0F1201C790E0007438F07F0A1220
:1002ED0001C790E000743890E000F01201C790E073
:1002FD0000743890E000F01201F390E0007406F005
:10030D001201F390E000740CF01201F390E0007410
:0E031D0001F01201F390E0007480F0F511225F
:0D032B0090E002E020E7F9EF90E001F02201
:030338000411802D
:01033B0000C1
:01033C00229E
:04033D00EE4F60130C
:100341007BEC7A02DBFEDAFC7C017DEDEF1F70ECC9
:040351001E80E922FF
:10035500758112E4787FF6D8FD900338E493700533
:1003650075A0FF805FC31392D5C31392D1FFA3E499
:1003750093F8B0D5403230D505E4A393F5F0E420E9
:10038500D102A39320D507F608DFF3A380CEC5835A
:10039500C5F0C583C582C8C582F0A3C583C5F0C5B0
:1003A50083C582C8C58280E1E8030303541F242066
:1003B500F9E85407F8E4D333B80002800333D8FDD5
:1003C50047F780C7758920758840759852758DE8FF
:0D03D50075A0FF90033CC082C083020404A9
:1003E20010AF0CC082C083C0E0E5A8C2E7800AC09B
:1003F20082C083C0E0E5A8D2E7900012F0A3E4F047
:100402008029C0E0E58730E206D0E01215A222D2B0
:10041200E2F5871213A77F00120F5EC2AFD0E0C0D1
:1004220082C083C0E09000137401F0D0E09000001D
:10043200F0A3E5F0F0A3E5D0F0A3D0E0F0A3D0E084
:10044200F0A3D0E0F0A3D0E0F0A3E581F075D000F6
:10045200A3E8F0A3E9F078027906A3E608F0D9FA56
:100462009000B8E06003020617900013E0700312D8
:100472000FAD7FA2121695020E041215FF90000A0C
:1004820078027906E0F608A3D9FA900008E0F8A30A
:10049200E0F9900007E0F581900006E0C0E09000EE
:1004A20005E0C0E0900000E0C0E0900013E0C0E092
:1004B200900001E0F5F0A3E0C0E0A3E0C0E0A3E01B
:1004C200F582D083D0D0D0E07005D0E0D2AF32D068
:1004D200E0D2AF2274FE2581F5817FA21216950229
:1004E2000E04900005E0FF7E007C01E4FD12009501
:1004F200900006E02FFFEE3400900010F0A3EFF022
:10050200020617C299C2ACC2BC900513C082C08356
:1005120032E4758107900000F5A8F5B8F587F58CEF
:10052200F58BF58DF58AF588F589F598F5F0F5D016
:0D05320014F580F590F5A0F5B0E402F0009E
:10053F0080FF820083008A008B008C0090FFA0FF59
:0E054F00A800B0FFB800D000E000F0000000EF
:10055D00900014EBF0A3EAF0A3E9F0E4A3F0740427
:10056D009000B5F0900014120082900017E0FD2D60
:10057D00FFE433FEE92FF9EA3EFA12004DFF7E004B
:10058D00900014120082900017E07C0025E0FD33EE
:10059D00E92DF9E43AFA09B900010A12004DFD12EC
:1005AD0008F290001475F0038001A3E0C0E0D5F0CF
:1005BD00F975F002900017E004F0A4FFD0E02FF8D9
:0D05CD00D0E035F0D005FC1200227098221D
:1005DA00E49000B8F0049000B9F0438704E4900076
:1005EA0005F0900006F07407900007F012161E122C
:0905FA0010721215F912047C22A2
:0A0603001210721215FC12047C2282
:0A060D001210721215F912047C227B
:10061700900006E0900018F0FF121695900018E081
:10062700FA900005E02A900018F0900005E0FF120C
:100637001695900018E0FA900007E02A900018F04D
:10064700900007E0FF121695900018E0F4FF0F12D4
:020657001695F6
:10065900E49000B4F012163DEF900019F09000B448
:10066900E070ED900019E0645560A3E064A5701096
:1006790012107274019000B8F01215F912047C225C
:07068900900019E0B45A1EB5
:10069000E49000B8F0121072900010E0FAA3E0FBB2
:0F06A0009000C5EAF0A3EBF0120FAD1204D622C2
:0106AF002228
:1006B0009000B3E06003E4FF2212163DEF90001AB1
:1006C000F09000B4E0600674019000B3F090001A5E
:0306D000E0FF2226
:1006D30090001BEEF0A3EFF09000B5E0B40403022A
:1006E30007F0500FE0602414602B14700302089786
:1006F3000208EFE024FA70030208A224FC7003024C
:0B07030008C71470030208DB0208EFB7
:10070E0090001B120078E493FF22E490001DF090FD
:10071E00001DE0FB2BFDE433FCED2412FFF582EC13
:10072E003416F583E493FA740193FBEA4B700302DB
:10073E0007E775F00290001DE0A4FBAAF02414F860
:10074E00F582E5F03416F583E49370087401937026
:04075E00030207E7A4
:1007620090001DE0FB2BFDE433FCED2412FFF5822B
:10077200EC3416F583E493FA740193FB90001BE0CA
:10078200B50205A3E0B50300405175F00290001DCB
:10079200E0A42414FDF582E5F03416F583E493C059
:1007A200E0740193C0E090001DE0FB2BFBE433FA00
:1007B200EB2412FCF582EA3416F583D00774019318
:1007C2002FFBD006E4933EFAF5F090001BE0B5F063
:1007D20005A3E0B503005003E4FF2290001DE024CE
:1007E20002F002071D90001B120078E0FF22900029
:1007F2001BE0FAA3E0FBBA0054B4A80280495011EE
:10080200EB247F601B14601E14602124FC60238093
:100812003CEB2430601F24F0602124F06023802D03
:10082200900007E0FF22900004E0FF22900003E026
:10083200FF22AF8722900002E0FF22900000E0FF3B
:1008420022900001E0FF22900012E0FF22E49000DB
:100852001DF090001DE0FB2410F582E43416F583B0
:04086200E493602893
:1008660090001BE0FCA3E0FDEB2410F582E43416B7
:10087600F583E493FBE4B50407EBB50503E4FF2237
:1008860090001DE004F080C690001CE0FF1216BB2D
:100896002290001CE0F890001B86072290001CE0C6
:1008A60025E0FB90001BE033FAEB2430F582EA34B6
:1008B6000BF583E493FA740193F5828A8312008B15
:1008C6002290001BE0FAA3E02412F582EA3416F522
:1008D60083E493FF2290001BE0FAA3E02410F58244
:0C08E600EA3416F583E493FF22E4FF22BD
:1008F20090001EEEF0A3EFF0A3EDF09000B5E060E3
:1009020018146024147003020A2424FE7003020ADD
:090912005F24FD7003020AD922E2
:10091B0090001EE0FEA3E0FFA3E0FD121602229062
:10092B000021E4F0A3F0900022E025E0FB900021F1
:10093B00E033FAEB2412F8F582EA3416F583E493EC
:10094B00FA740193FBEA4B7003020A16900022E043
:10095B00FB900021E0FAEBC333CA33CAFB2414F833
:10096B00EA3416F5838882E493700874019370035C
:03097B00020A1657
:10097E00900022E025E0FB900021E033FAEB2412F8
:10098E00F8F582EA3416F583E493FA740193FB903A
:10099E00001EE0FCA3E0FDECB50204EDB503004043
:1009AE0053900022E0FB900021E0FAEBC333CA33F0
:1009BE00CA2414FCEA3416F5838C82E493FE740187
:1009CE0093FF900022E025E0FB900021E033FAEB4C
:1009DE002412FDF582EA3416F5837401932FFFE499
:1009EE00933EFEF5F090001EE0B5F005A3E0B507CE
:1009FE0000500122900022E02402FB900021E034FE
:100A0E0000F0A3EBF0020931900020E0FA90001EF6
:100A1E00120078EAF022900020E0FA90001FE09099
:100A2E00001EF8A602E0B40006A3E0B40701D350FE
:100A3E001F900002E054187017900020E0FA90000A
:100A4E001EE0FCA3E02408F582EC3400F583EAF006
:100A5E002290001EE0FAA3E0FBBA0062B4A8028066
:100A6E0054500DEB247F601714601D146023804ECC
:0F0A7E00EB2430602524F0602A24F0602F803FA5
:100A8D00900020E0900007F022900020E0900004FC
:100A9D00F022900020E0900003F022900020E090E2
:100AAD000002F022900020E0900000F02290002043
:100ABD00E0900001F022900020E0900012F02290D2
:100ACD00001EA3E0FFA3E0FD1216C72290001EE05A
:0B0ADD00FEA3E0FFA3E0FD1212852243
:060AE800900000E0FF2277
:060AEE00900001E0FF2270
:060AF400900008E0FF2263
:060AFA00900009E0FF225C
:060B000090000AE0FF2254
:060B060090000BE0FF224D
:060B0C0090000CE0FF2246
:060B120090000DE0FF223F
:060B180090000EE0FF2238
:060B1E0090000FE0FF2231
:060B2400900005E0FF2235
:060B2A00900006E0FF222E
:100B30000AE80AEE0AF40AFA0B000B060B0C0B1279
:080B40000B180B1E0B240B2AFD
:100B480005DA050506AF06AF060304E406AF060D91
:070B580074349000C3F02289
:100B5F007B027A0079BA12004D540F9000B5F090D5
:100B6F0000CBF09000BCE0FAA3E0FBA3EAF0A3EB0C
:100B7F00F09000BA7A00E054807003020D127B02ED
:0A0B8F0012004D54706003020D12B5
:0A0B99009000C0E0700AA3E07006AF
:100BA3007FD0121695229000C7E4F0A3F09000C006
:100BB300E0FAA3E024FFFFEA34FFFEE4FC7D8C129D
:100BC30000D19000C7E0B50606A3E0B50701D34006
:040BD30003020DFE0E
:100BD7009000C7E0B506078FF0A3E06F600B9000A9
:100BE70023E4F0A3748CF080179000C0E0FEA3E02C
:100BF700FFE4FC7D8C1200D1EC900023F0A3EDF014
:100C0700900023E0700DA3E07009900023E4F0A3A7
:100C1700748CF07F3A121695900023E0FF9000BB8A
:100C2700F0121695900023A3E0FF1216959000BBD3
:100C3700E0FC900023A3E02C9000BBF09000BEE006
:100C4700FAA3E0FB9000C9EAF0A3EBF0900023E0E1
:100C5700FAA3E0FB9000BFE02BFB9000BEE03AF563
:100C6700F09000C9E0FCFEA3E0FDFFECB5F004ED59
:050C7700B50300502947
:100C7C001206D3EF9000C2F01216959000BBE0FA6A
:100C8C009000C2E02A9000BBF09000CAE004F09003
:100C9C0000C970B3E004F080AE9000BBE0F4FF0F2D
:100CAC001216951206B0EFFB9000CCF07A00EF64B0
:100CBC00A57016900023E0FAA3E0FB9000BFE02B98
:100CCC00F09000BEE03AF080299000CCE0FB7A0076
:040CDC0064A070118F
:100CE0009000C8E014F0F49000C77012E014F08097
:100CF0000D9000CCE0FBE4B47504BB300122900001
:100D0000C8E004F09000C76003020BB0E004F002FA
:100D10000BB09000BAE05440607C7B027A0079BA54
:070D200012004D54B0706F8A
:100D27009000CD7400F0A37427F09000C9E4F0A3FD
:100D37007402F09000B6E0FCA3E0FD9000C9E0FA71
:100D4700A3E0FBEAB50404EBB505004003020DFE82
:100D57009000BEE0FEA3E0FF9000CD120078E0FD1A
:100D67001208F29000BFE004F09000BE7003E004A8
:100D7700F09000CEE004F09000CD7003E004F09016
:0F0D870000CAE004F09000C970A9E004F080A455
:100D96009000BAE05420605B7B027A0079BA1200B8
:050DA6004D54D0704E19
:100DAB007F311216959000C4E0700E9000CBE0647A
:030DBB00036006CC
:100DBE007FAA121695229000CBE0B40801D340070B
:070DCE007FC0121695802979
:100DD5009000B9E070179000CBE0FA2A900B48FC20
:100DE50093CC0493F5828C8312008B800CE49000E5
:0F0DF500B9F080057FC01216957FA212169522C5
:020E0400C2AF7B
:100E060074019000B4F09000B4E0600A12163DEF51
:100E16009000C2F080F0E49000B3F09000C2E0646D
:0F0E2600A07005120B5F80D89000C2E0B4551A7F
:100E35009000C4E070077FAA12169580057FA21264
:100E4500169574019000C4F080B79000C2E0B43AE2
:060E5500028003020F4DB4
:100E5B001206B0EF79BA7A007B021200061206B0C6
:100E6B00EF9000B6F0A3E4F01206B09000B7E02FBD
:100E7B00F09000B6E03400F0FBA3E02BFC79BA7ADB
:100E8B00007B0212004D2C9000BBF09000B6E0707E
:100E9B0004A3E0604F9000CFE4F0A3F09000B6E025
:100EAB00F5F0A3E0FB9000CFE0B5F005A3E0B503B0
:030EBB00005031B3
:100EBE001206B0EF9000D1F09000D0E02425FA9009
:100ECE0000CFE03400F5838A82EFF09000BBE02F74
:010EDE00F023
:100EDF009000D0E004F09000CF70BDE004F080B837
:100EEF009000BBE0C0E01206B0D0E02F9000BBF046
:100EFF00900025E0FAA3E0FDE42DFDE43A9000BC5C
:100F0F00F0A3EDF0900027E0FAA3E0FDE42DFDE45F
:100F1F003A9000C0F0A3EDF09000BBE0700B900092
:100F2F00B3E07005120B5F80239000B3E060077F82
:100F3F00B012169580167FE0121695020E069000DD
:0F0F4F00C2E07003020E067FA0121695020E0676
:080F5E009000D2EFF0EF703CAF
:100F6600120B58E49000B3F0049000C4F0E4900033
:100F7600B8F0A3F07B027A0079BA1200069000BBA3
:100F8600F09000BEF0A3F0A3F0A3F0A3F09000C58C
:0C0F9600F0A3F01211D27FAA12169522CF
:0B0FA200E49000B3F07FA2121695222D
:100FAD00900005E0FAE4FB900006E0FDE42DFDE481
:100FBD003AFCED24FDFDEC34FF9000D3F0A3EDF0F1
:100FCD009000D3E0FEA3E0FFE4FD121184EF90004A
:100FDD00D5F090115DE493F5F09000D5E065F060EB
:0F0FED001E9000D3E0FEA3E0FF1211F4EF60109E
:100FFC009000D3E0900005F09000D4E0900006F053
:10100C009000C5E0FEA3E0FFE4FDFB121184EF901D
:10101C0000D5F090115DE493F5F09000D5E065F00B
:02102C0060431F
:10102E00E49000B5F09000C5E0FEA3E0FF90160D31
:10103E00E493FD1208F29000C5E0FAA3E02401FF4C
:10104E00E43AFE90160EE493FD1208F29000C6E00C
:10105E002402FF9000C5E03400FE90160FE493FDCD
:04106E001208F22250
:10107200900005E0FA900006E0FDE42DFDE43A90D0
:1010820000C5F0A3EDF09000C5E0B40005A3E0B404
:10109200020050099000D6E4F0A3F080149000C63C
:1010A200E024FEFB9000C5E034FF9000D6F0A3EBF5
:0110B200F04D
:1010B3009000D6E0FEA3E0FFE4FDFB121184EF9065
:1010C30000D8F090115DE493FAF5F09000D8E06554
:0310D300F0605B6F
:1010D600E49000B5F09000D6E0FAA3E0FB9000C5DE
:1010E600EAF0A3EBF0E49000D9F09000C5E0FCA391
:1010F600E0FD9000D9E0FBED2BFFE43CFEE0FB9029
:1011060000D8E075F005A424DCF582E5F03400F59E
:1011160083EB2582F582E43583F583E0FD1208F240
:101126009000D9E004F0B403C180289000D7E00411
:10113600F09000D67003E004F09000C5E0FAA3E05A
:10114600FB9000D6E0B50206A3E0B50301D3500339
:071156000210B31215EB2299
:01115D008011
:10115E007E00EE75F005A424DAF582E5F03400F594
:10116E0083E0B4FF08A3E0B4FF038E07220EEE6403
:06117E008070DF7F80227B
:1011840090035BEEF0A3EFF0A3EDF0ED6002803B83
:10119400E490035EF090035BE0FEA3E0FF90035E47
:1011A400E075F005A424DAF582E5F03400F583E077
:1011B400B5060BA3E0B5070690035EE0FF2290039B
:0E11C4005EE004F0648070CD7F80227F802288
:0211D2007F009C
:1011D400EF75F005A424DAF582E5F03400F58374A4
:1011E400FFF0A3F00FEF648070E6E490035AF0225E
:1011F40090035FEEF0A3EFF0E49000B5F090160DCD
:1012040093FB7A00C002C0031206D3EFFDD007D0CF
:10121400F0E4B5F0068FF0ED6F6003E4FF22901662
:101224000EE493FB7A00C002C003900360E0240143
:10123400FF90035FE03400FE1206D3EFFDD007D029
:10124400F0E4B5F0068FF0ED6F6003E4FF22901632
:101254000FE493FB7A00C002C003900360E0240211
:10126400FF90035FE03400FE1206D3EFFDD007D0F9
:10127400F0E4B5F0068FF0ED6F6003E4FF227F0128
:011284002247
:0E128500900361EEF0A3EFF0A3EDF0ED7076B4
:10129300E4FDFB121184EF900364F0EF648060655A
:1012A300E49000B5F0900365F0900361E0FCA3E0E7
:1012B300FD900365E0FBED2BFFE43CFEE0FB9003B8
:1012C30064E075F005A424DCF582E5F03400F583D1
:1012D300EB2582F582E43583F583E0FD1216029057
:1012E3000365E004F0B403C1900364E075F005A462
:1012F30024DAF582E5F03400F58374FFF0A3F0906F
:06130300035AE014F02281
:1013090012115EEF900364F0EF648070030213A67C
:10131900900361E0FCA3E0FDEF75F005A424DAF584
:1013290082E5F03400F583ECF0A3EDF0E49000B52C
:05133900F0900365F0D7
:10133E00900361E0FCA3E0FD900365E0FBED2BFF65
:10134E00E43CFE1206D3900365E0FB900364E07567
:10135E00F005A424DCF582E5F03400F583EB25825C
:10136E00F582E43583F583EFF0900362E02BFF9076
:10137E000361E03400FE900365E0240DF582E43451
:10138E0016F583E493FD121602900365E004F0B4A3
:09139E00039E90035AE004F022C2
:1013A70090036674F8F0A3E4F0A374FCF0A3E4F0F0
:1013B700900368E0FEA3E02400FF8E838F82F09005
:1013C7000366E0FEA3E02402FF8E838F82741AF087
:1013D70000000000000000000000742AF000000078
:1013E70000000000000000743AF000000000000058
:1013F70000000000744AF000000000000000000038
:1014070000745AF000000000000000000000740A99
:10141700F0900366E0FEA3E02401FF8E838F82E055
:10142700FC900366E0FEA3E02402FF8E838F8274A4
:1014370005F0900366E0FEA3E02404FF8E838F820D
:101447007488F0900366E0FEA3E02400FF8E838F8C
:10145700827413F07407F0900366E0FEA3E02401A2
:10146700FF8E838F82E0FFE42C2F24F4601F90030C
:101477006674C0F0A3E4F0A374A0F0A3E4F09003B3
:1014870068E0FEA3E02400FF8E838F82F09003665E
:10149700E0FEA3E02400FF8E838F827413F07407AD
:1014A700F07407B40114900366E0FEA3E02401FF83
:1014B7008E838F827488F002156FB40214900366CE
:1014C700E0FEA3E02401FF8E838F827499F002155A
:1014D7006FB40314900366E0FEA3E02401FF8E833C
:1014E7008F8274BBF002156FB40413900366E0FE9D
:1014F700A3E02401FF8E838F8274CCF0806AB40549
:1015070022900366E0FEA3E02402FF8E838F82E031
:10151700900366E0FEA3E02401FF8E838F8274446C
:10152700F08045B40622900366E0FEA3E02402FFA4
:101537008E838F82E0900366E0FEA3E02401FF8E96
:10154700838F827488F08020900366E0FEA3E024F6
:1015570002FF8E838F82E0900366E0FEA3E0240102
:10156700FF8E838F827466F0900366E0FEA3E0240B
:1015770004FF8E838F827488F0900366E0FEA3E0F9
:101587002402FF8E838F827405F0900366E0FEA32A
:10159700E02405FF8E838F827404F0D2889003665F
:1015A700E0B4F83F7F127E167DF81216027F137E95
:1015B700167D001216027F147E167D081216027F12
:1015C700157E167D001216027F167E167D001216F6
:1015D700027F177E167D001216027F187E167D0089
:1015E70012160222D2A8D2B8222089037F00227FB6
:0B15F7000122D28922C28922D2A82240
:0E160200C2B78E838F82EDF0D2B722D289005C
:0E1610009900A0001000C000100000000000B3
:10161E009000057400F09000067400F090000074C5
:0F162E00FFF590F5B0E4F58AF58CF5D0F5F022D4
:07163D00E4FCFD9000B4F095
:0B1644000DED70010CBC750CBD3009F1
:10164F0074019000B4F0E4FF22900366E0B4C00E82
:10165F00A3E0B4000990C001E0FB7A00800590F888
:10166F0001E0FBEB30E0CE900366E0B4C00EA3E0E8
:10167F00B4000990C003E0FB7A00800790F803E004
:06168F00FB7A008B07222C
:0C169500900366E0B4C012A3E0B4000DA6
:0D16A100EF90C003F090C001E030E2F922AC
:0D16AE00EF90F803F090F801E030E2F9222F
:1016BB00EFFD7E167FC5121602AF8022EDC0E0EF64
:0E16CB00FD7E167FD7121602D0E0FF8F802220
:00000001FF
